:020000040000FA
:0A000000000000008FEF00F09DD01B
:08001800EAD00E6E960E056E93
:10002000980E066E55D8D8B4CA90D8A4CA80FC0FD2
:10003000D8A0CA92D8B0CA82800E056E960E066EFF
:10004000980E096E0A6ACAB025D8CAB223D842D817
:100050000504CB6E05C007F006C008F000500B6E1B
:100060000C6E003C0C6A4BD80A500E2E0AD0BE6EA5
:100070000C0EBD6E09BEBD8A09BCBD889394CA84AE
:100080001200BB6E0C0EBA6E09BEBA8A09BCBA88E1
:100090009492F5D700D8D890093206320532120072
:1000A000086A076EFF0E0726082200D0D8A01200AB
:1000B000030E066EE60E02D8F5D7066AFE0F056E31
:1000C000E86A065AD8A012000000050600D0F8D74A
:1000D0000A6A096A100EF36E063409360A360750AA
:1000E000095C08500A5805E30750095E08500A5A8F
:1000F000D88005360636F32EEFD70550120007508C
:100100000B02F3CF09F0F4CF0AF008500B02F350C2
:100110000A2607500C02F3500A26095012004F0E0F
:10012000AF6E240EAC6E900EAB6E0001C69A430EFD
:10013000926EE00E936EC00E946E0F0EC16E070E9F
:10014000B46E6CD0F2A403D0F294817A11009EAA0E
:1001500019D0060EAB1412E1E2CF43F0E1CF42F02A
:10016000442A10EE4EF04450E126000EE222AECFBB
:10017000E7FF43C0E2FF42C0E1FF1100AE50AE50C6
:10018000AB98AB8811004450455C14E0452AEACF97
:1001900006F0E9CF05F000EE4EF04550E926000EDE
:1001A000EA22EF50056E06C0EAFF05C0E9FFD880DD
:1001B000120004D0E868056ED8A012001200446A4C
:1001C000456A9D8A9F8AF28EF28C12009D9A00EEFB
:1001D0004EF0010EF46EF36AF306000EF45AEE6A66
:1001E000F450F310F9E1446A456A9D8A1200F29EC8
:1001F000E0CF4EF3D8CF4FF3E8CF50F3F28E0001AB
:10020000A192F29E4EC3E0FF4FC3D8FF50C3E8FF58
:10021000F28E10009EA8FED7AD6E120094928B92C3
:10022000929A899A9298899892968996939A8A9A9C
:10023000949A8B9A94988B9893948A94256A306AAE
:100240002C682D6A66EC04F066EC06F0E6C122F03C
:10025000E7C123F0200E216E206A205022242A6E4E
:10026000215023202B6E4C0E2F6E2DC000F02BC082
:1002700008F02AC007F0010ED0DE2CC000F02BC021
:1002800008F02AC007F0020EC8DE939A8A8A320E5E
:1002900007DF939A8A9A246A296A91DF97DFCD6AE9
:1002A000F294F28A870ED56EB16AA192A082B36AE7
:1002B000B26AD08EA292B00EB16E00EE46F0080E79
:1002C000EE68E82EFDD74168408E3A6A396A386A8E
:1002D000376A3B2AE86A3BB2010F3CB0010806E1ED
:1002E0003C70372A000E382239223A224CDF116E38
:1002F000EA0E115C07E3FE0E115C02E339D102D075
:10030000136A36D111AE37D0136A890E115C05E13C
:1003100011C013F0146815682DD0990E115C05E119
:1003200011C013F01668176825D0A90E115C05E1FD
:1003300011C013F0186819681DD0B90E115C05E1E1
:1003400011C013F01A681B6815D0C90E115C04E1C6
:1003500011C013F01C680ED0D90E115C04E111C05D
:1003600013F01D6807D0E90E115C04E111C013F011
:100370001E681F68FCD0135202E1FAD0F8D0890E33
:10038000135C19E1142803E111C014F012D0780EA7
:10039000145C04E189982990249009D0790E145CAA
:1003A00004E189962992249202D01468E1D014685D
:1003B000DED0DED0DCD0990E135CD8A47CD0162819
:1003C00003E111C016F075D011C017F0175212E1F9
:1003D000780E165C04E189982990249009D0790E52
:1003E000165C04E189962992249202D01668C0D046
:1003F0001668BDD02552D8B45CD0780E165C29E1C1
:1004000089887F0E175C22E202EE4EF0D8901734F6
:10041000E926000EEA22EECF31F0EFCF32F0248051
:1004200031503724016E32503820026E000E3920D0
:10043000036E000E3A20046E04C049F003C048F079
:1004400002C047F001C046F0298002D024902980E4
:100450002ED0790E165C29E189867F0E175C22E288
:1004600002EE4EF0D8901734E926000EEA22EECFC5
:1004700033F0EFCF34F0248233503724016E345000
:100480003820026E000E3920036E000E3A20046EF2
:1004900004C04DF003C04CF002C04BF001C04AF064
:1004A000298202D02492298202D0166861D016686F
:1004B0005ED05ED05CD0A90E135C36E1182804E152
:1004C00011C018F055D02FD0780E185C14E111C06F
:1004D00035F035520CE002EE4EF0D8903534E92676
:1004E000000EEA22EECF31F0EFCF32F003D0326AC5
:1004F000316A299016D0790E185C13E111C036F0DC
:1005000036520CE002EE4EF0D8903634E926000E5A
:10051000EA22EECF33F0EFCF34F003D0346A336AFF
:100520002992186825D023D0B90E135C0AE11A2845
:1005300003E111C01AF003D011C01BF0F3D818D09A
:1005400016D0C90E135C07E11C2803E111C01CF092
:10055000C2D80ED00CD0E90E135C09E11E2803E1CD
:1005600011C01EF003D011C01FF0B7D801D079D848
:10057000020E415CD8B06DD03D50375C3E503858CB
:100580003F50395840503A58D8A044D0408E41523C
:100590001FE129B007D024908998496848684768C6
:1005A000466815D0807831503724016E325038209B
:1005B000026E000E3920036E000E3A20046E04C055
:1005C00049F003C048F002C047F001C046F021D016
:1005D000010E415C1EE129B207D0249289964D6834
:1005E0004C684B684A6815D0807633503724016ECA
:1005F00034503820026E000E3920036E000E3A206F
:10060000046E04C04DF003C04CF002C04BF001C0BA
:100610004AF027D83AAE1CD03A6A396A386A376A43
:10062000246A296A00EE46F0080EEE68E82EFDD72F
:10063000006A2BC008F02AC007F0010E0DEC00F094
:1006400000682BC008F02AC007F0020E0DEC00F085
:1006500006D03AAE04D03A6A396A386A376A81708D
:1006600038D64168408E126A020E125C33E2D8908E
:100670001234E96EEA6AEA36E936EA36460EE926C7
:10068000000EEA22EFCF01F0ECCF02F0ECCF03F046
:10069000ECCF04F03D50015C3E5002583F500358EF
:1006A0004050045815E2D8901234E96EEA6AEA36EE
:1006B000E936EA36460EE926000EEA22EFCF3DF093
:1006C000ECCF3EF0ECCF3FF0ECCF40F012C041F069
:1006D000122ACAE312001C681200D8901F30216E43
:1006E000206A20321E502026000E21222050222473
:1006F0002A6E215023202B6E2CC000F02BC008F056
:100700002AC007F0020E0DEC00F02DC000F02BC047
:1007100008F02AC007F0010E0DEC00F01E68120070
:100720001D681200070E1A5C14E11B5202E12C68CE
:1007300006D0D8901B342C6E2C50FE082C6E2CC08A
:1007400000F02BC008F02AC007F0020E0DEC00F0FC
:100750008AD0080E1A5C0CE11BC02DF02DC000F0F1
:100760002BC008F02AC007F0010E0DEC00F07BD082
:100770001E0E1A5C25E11B5208E1296A326A316AB1
:10078000356A346A336A366A1AD01BC035F002EE15
:100790004EF0D8901B34E926000EEA22EECF31F05D
:1007A000EFCF32F01BC036F002EE4EF0D8901B3483
:1007B000E926000EEA22EECF33F0EFCF34F053D02B
:1007C0001F0E1A5C31E101EE4EF0D8901B34E92681
:1007D000000EEA22EECF22F0EFCF23F03E0E235C94
:1007E00007E303E1810E225C03E38A84000101D068
:1007F0008A94205022242A6E215023202B6E1BC065
:100800002FF02CC000F02BC008F02AC007F0020E19
:100810000DEC00F02DC000F02BC008F02AC007F04E
:10082000010E0DEC00F01FD0410E1A5C0DE11B52C1
:1008300004E1899A8B98306A06D0255204E0898AAF
:100840001BC030F08B880FD0420E1A5C08E11B529F
:1008500003E110D8256A02D08B8A256804D07B0E6C
:100860001A5CD8B402D81A681200246A899889964A
:10087000296A1200246A89988996296A2C682D6A47
:100880002F6AE6C122F0E7C123F0200E216E206A14
:10089000205022242A6E215023202B6E2DC000F0E0
:1008A0002BC008F02AC007F0010E0DEC00F02CC0A0
:1008B00000F02BC008F02AC007F0020E0DEC00F08B
:1008C0008A848B9A306A899A8B98120002014F6948
:1008D0004E69A20E516FC30E506F9A0E536F460EA3
:1008E000526F960E556F320E546F920E576F3A0E2E
:1008F000566F8E0E596F5D0E586F8A0E5B6F9A0E93
:100900005A6F860E5D6FF00E5C6F830E5F6F5F0E29
:100910005E6F7F0E616FE70E606F7C0E636F850EFA
:10092000626F790E656F3B0E646F760E676F070E10
:10093000666F720E696FE80E686F6F0E6B6FDF0E79
:100940006A6F6C0E6D6FEA0E6C6F6A0E6F6F0A0E37
:100950006E6F670E716F3C0E706F640E736F820E58
:10096000726F610E756FDA0E746F5F0E776F440EE3
:10097000766F5C0E796FBF0E786F5A0E7B6F4C0EE0
:100980007A6F570E7D6FE90E7C6F550E7F6F960E56
:100990007E6F530E816F806F510E836F200E826FBA
:1009A0004E0E856FFB0E846F4C0E876FE50E866FC3
:1009B0004A0E896FDC0E886F480E8B6FE20E8A6FCD
:1009C000460E8D6FF50E8C6F450E8F6F150E8E6F68
:1009D000430E916F420E906F410E936F7B0E926F9C
:1009E0003F0E956FC00E946F3E0E976F100E966F70
:1009F0003C0E996F6D0E986F3A0E9B6FD40E9A6FE6
:100A0000390E9D6F460E9C6F370E9F6FC20E9E6F04
:100A1000360EA16F490EA06F340EA36FDA0EA26FCF
:100A2000330EA56F740EA46F320EA76F180EA66F4B
:100A3000300EA96FC50EA86F2F0EAB6F7B0EAA6F7D
:100A40002E0EAD6F3A0EAC6F2D0EAF6F020EAE6F65
:100A50002B0EB16FD10EB06F2A0EB36FA90EB26F0D
:100A6000290EB56F880EB46F280EB76F6F0EB66F74
:100A7000270EB96F5E0EB86F260EBB6F530EBA6F9E
:100A8000250EBD6F500EBC6F240EBF6F540EBE6F8F
:100A9000230EC16F5E0EC06F220EC36F6F0EC26F4A
:100AA000210EC56F860EC46F200EC76FA30EC66FD2
:100AB0001F0EC96FC60EC86F1E0ECB6FEF0ECA6F2A
:100AC0001E0ECD6FCC6F1D0ECF6F520ECE6F1C0E53
:100AD000D16F8C0ED06F1B0ED36FCB0ED26F1B0E4F
:100AE000D56F0F0ED46F1A0ED76F580ED66F190E22
:100AF000D96FA50ED86F180EDB6FF80EDA6F180ECF
:100B0000DD6F4F0EDC6F170EDF6FAB0EDE6F170E53
:100B1000E16F0A0EE06F160EE36F6F0EE26F150EB7
:100B2000E56FD70EE46F150EE76F430EE66F140EF8
:100B3000E96FB30EE86F140EEB6F270EEA6F130E1A
:100B4000ED6F9F0EEC6F130EEF6F1A0EEE6F120E1D
:100B5000F16F990EF06F120EF36F1B0EF26F110E04
:100B6000F56FA10EF46F110EF76F290EF66F100ED0
:100B7000F96FB50EF86F100EFB6F440EFA6F0F0E83
:100B8000FD6FD60EFC6F0F0EFF6F6B0EFE6F0F0E1C
:100B90000301016F030E006F0E0E036F9D0E026FB7
:100BA0000E0E056F3A0E046F0D0E076FDA0E066F0C
:100BB0000D0E096F7C0E086F0D0E0B6F210E0A6F64
:100BC0000C0E0D6FC80E0C6F0C0E0F6F720E0E6FA9
:100BD0000C0E116F1E0E106F0B0E136FCC0E126FDA
:100BE0000B0E156F7C0E146F0B0E176F2E0E166FFB
:100BF0000A0E196FE30E186F0A0E1B6F990E1A6F0B
:100C00000A0E1D6F510E1C6F0A0E1F6F0B0E1E6F0A
:100C1000090E216FC80E206F090E236F850E226FFB
:100C2000090E256F450E246F090E276F060E266FDD
:100C3000080E296FC90E286F080E2B6F8E0E2A6FB3
:100C4000080E2D6F540E2C6F080E2F6F1C0E2E6F7A
:100C5000070E316FE50E306F070E336FAF0E326F38
:100C6000070E356F7B0E346F070E376F490E366FE8
:100C7000070E396F170E386F060E3B6FE70E3A6F8F
:100C8000060E3D6FB90E3C6F060E3F6F8B0E3E6F2A
:100C9000060E416F5F0E406F060E436F340E426FBB
:100CA000060E456F0A0E446F050E476FE10E466F44
:100CB000050E496FB90E486F050E4B6F930E4A6FC4
:100CC000050E4D6F6D0E4C6F00011200126A270E5B
:100CD000125C0DE201EE4EF0D8901234E926000EBF
:100CE000EA22680EEE6E520EEF6E122AF0E3090E43
:100CF00001019D6FB90E9C6F0A0E9F6F4D0E9E6F86
:100D00000A0EA16FE90EA06F0B0EA36F5E0EA26F0D
:100D10000C0EA56F400EA46F0C0EA76FFA0EA66FF7
:100D20000E0EA96F240EA86F0E0EAB6F910EAA6F58
:100D30000F0EAD6F3D0EAC6F100EAF6F5A0EAE6F53
:100D4000110EB16F530EB06F120EB36F5A0EB26F19
:100D5000130EB56F720EB46F140EB76F9A0EB66F96
:100D6000150EB96FD30EB86F160EBB6FBC0EBA6FEF
:100D7000180EBD6F800EBC6F190EBF6FF40EBE6FE4
:100D80001B0EC16F800EC06F1D0EC36F220EC26F8F
:100D90001E0EC56F7A0EC46F200EC76FB40EC66FDD
:100DA000220EC96FA60EC86F240ECB6FB50ECA6F88
:100DB000260ECD6FE40ECC6F290ECF6F340ECE6FA2
:100DC0002B0ED16FA70ED06F2E0ED36F400ED26FA9
:100DD000310ED56FD46B330ED76FE90ED66F370E49
:100DE000D96FD86B3A0EDB6F450EDA6F3D0EDD6FB3
:100DF000BC0EDC6F410EDF6F680EDE6F450EE16FDB
:100E00004B0EE06F490EE36F6A0EE26F4D0EE56F19
:100E1000C80EE46F520EE76F680EE66F4D0E126E4D
:100E20000001800E125C0DE201EE4EF0D8901234FB
:100E3000E926000EEA22680EEE6E520EEF6E122ABE
:080E4000EFE312001200FFD7DE
:020000040030CA
:0300010006160ED2
:020005008580F4
:060008000FC00FE00F40E5
:00000001FF
